:020000040000FA
:04080000E7EF07F027
:1008100003B213EF05F0F2B42EEF05F09EB036EF01
:1008200005F09EB23EEF05F0F2A81AEF04F0F2B226
:1008300025EF04F0F2A620EF04F0F2B022EF04F06E
:1008400096EF07F0F296F290FF00CD90F2929EA004
:100850002FEF04F00101533F2FEF04F0542BAEC1F2
:10086000B2F1AFC1B3F1B0C1B4F1B1C1B5F1AAC138
:10087000AEF1ABC1AFF1ACC1B0F1ADC1B1F1A6C148
:10088000AAF1A7C1ABF1A8C1ACF1A9C1ADF1A2C158
:10089000A6F1A3C1A7F1A4C1A8F1A5C1A9F19EC168
:1008A000A2F19FC1A3F1A0C1A4F1A1C1A5F19AC178
:1008B0009EF19BC19FF19CC1A0F19DC1A1F196C188
:1008C0009AF197C19BF198C19CF199C19DF1CECF4E
:1008D00096F1CFCF97F153C198F154C199F1CF6AF6
:1008E000CE6A0101536B546B9E90CD800FBC0F8E6E
:1008F0000FBA7EEF04F00F8A96EF07F00F8C0FBE51
:10090000BAEF04F096C19AF197C19BF198C19CF19E
:1009100099C19DF19AC19EF19BC19FF19CC1A0F12B
:100920009DC1A1F19EC1A2F19FC1A3F1A0C1A4F1FB
:10093000A1C1A5F1A2C1A6F1A3C1A7F1A4C1A8F1CB
:10094000A5C1A9F1A6C1AAF1A7C1ABF1A8C1ACF19B
:10095000A9C1ADF1AAC1AEF1ABC1AFF1ACC1B0F16B
:10096000ADC1B1F1AEC1B2F1AFC1B3F1B0C1B4F13B
:10097000B1C1B5F101015E6B5F6B606B616B96514C
:100980005E2797515F2398516023995161239A51B3
:100990005E279B515F239C5160239D5161239E5193
:1009A0005E279F515F23A0516023A1516123A25173
:1009B0005E27A3515F23A4516023A5516123A65153
:1009C0005E27A7515F23A8516023A9516123AA5133
:1009D0005E27AB515F23AC516023AD516123AE5113
:1009E0005E27AF515F23B0516023B1516123B251F3
:1009F0005E27B3515F23B4516023B5516123D89072
:100A00000101613360335F335E33D890010161339C
:100A100060335F335E33D8900101613360335F33FD
:100A20005E3396EF07F00392030103EE00F080516E
:100A30007F0BE92604C0EFFF802B8151805D700B96
:100A4000D8A48B8200008051815D700BD8A48B925A
:100A500081518019D8B4079096EF07F0F294010104
:100A6000453F96EF07F0462B96EF07F09E90010169
:100A7000533F96EF07F0542B96EF07F09E92040039
:100A800062A143EF05F0077C07AC5EEF05F0C2748E
:100A9000C2B458EF05F0C3CFB3F5C4CFB4F5050128
:100AA000D890B433B333D890B433B3335FEF05F099
:100AB000C3CF55F1C4CF56F15FEF05F0C28207B442
:100AC000CCEF05F047C14BF148C14CF149C14DF1A4
:100AD0004AC14EF15EC162F15FC163F160C164F170
:100AE00061C165F196C1B6F197C1B7F198C1B8F18E
:100AF00099C1B9F19AC1BAF19BC1BBF19CC1BCF1DA
:100B00009DC1BDF19EC1BEF19FC1BFF1A0C1C0F1A9
:100B1000A1C1C1F1A2C1C2F1A3C1C3F1A4C1C4F179
:100B2000A5C1C5F1A6C1C6F1A7C1C7F1A8C1C8F149
:100B3000A9C1C9F1AAC1CAF1ABC1CBF1ACC1CCF119
:100B4000ADC1CDF1AEC1CEF1AFC1CFF1B0C1D0F1E9
:100B5000B1C1D1F1B2C1D2F1B3C1D3F1B4C1D4F1B9
:100B6000B5C1D5F1B3C5B5F5B4C5B6F5B5C5B7F5DD
:100B7000B6C5B8F5010155515B2756515C23E86AAB
:100B80005D230E2ECCEF05F05CC157F15DC158F12D
:100B90005B6B5C6B5D6B078E0201002F96EF07F0BD
:100BA0003C0E006F00C10CF101C10DF102C10EF14C
:100BB00003C10FF104C110F105C111F106C112F119
:100BC00007C113F108C114F109C115F10AC116F1E9
:100BD0000BC117F134C135F105012F51000AD8B40A
:100BE00095EF06F005012F51010AD8B41FEF06F06A
:100BF00005012F51020AD8B460EF06F005012F510C
:100C0000030AD8B460EF06F005012F51040AD8B4E6
:100C100060EF06F005012F51050AD8B460EF06F029
:100C200005012F51060AD8B460EF06F005012F51D7
:100C3000070AD8B460EF06F02F6B95EF06F00501B8
:100C400053672AEF06F054672AEF06F055672AEF3C
:100C500006F056672EEF06F095EF06F057C500F147
:100C600058C501F159C502F15AC503F10101010E40
:100C7000046F000E056F000E066F000E076F5FEC2D
:100C80001FF000C157F501C158F502C159F503C164
:100C90005AF5006753EF06F0016753EF06F002675D
:100CA00053EF06F0036795EF06F053C557F554C5AB
:100CB00058F555C559F556C55AF50F8895EF06F004
:100CC0000501306766EF06F095EF06F00FBE7BEF8B
:100CD00006F010A080EF06F00101476777EF06F0FD
:100CE000486777EF06F0496777EF06F04A677BEFD2
:100CF00006F080EF06F007AE80EF06F092EF06F008
:100D00000501312F95EF06F03C0E316F302F95EF36
:100D100006F00101000E626FE00E636FA50E646FB6
:100D2000010E656F0501306B0F880501626B33B7EB
:100D30009BEF06F062810CC100F10DC101F10EC103
:100D400002F10FC103F110C104F111C105F112C18B
:100D500006F113C107F114C108F115C109F116C15B
:100D60000AF117C10BF135C134F100C10CF101C119
:100D70000DF102C10EF103C10FF104C110F105C163
:100D800011F106C112F107C113F108C114F109C133
:100D900015F10AC116F10BC117F134C135F101018A
:100DA0008A67DAEF06F08B67DAEF06F08C67DAEF26
:100DB00006F08D67DEEF06F00EEF07F08EC100F152
:100DC0008FC101F190C102F191C103F10101010E46
:100DD000046F000E056F000E066F000E076F5FECCC
:100DE0001FF000C18EF101C18FF102C190F103C16A
:100DF00091F1006703EF07F0016703EF07F0026767
:100E000003EF07F003670EEF07F08AC18EF18BC185
:100E10008FF18CC190F18DC191F10F80D57ED5BE3F
:100E200069D0D6CF47F1D7CF48F145C149F1E86A3B
:100E3000E8CF4AF1109047C100F148C101F149C122
:100E400002F14AC103F101010A0E046F000E056FA1
:100E5000000E066F000E076F5FEC1FF000AF1080F2
:100E6000010154A740EF07F00F9A0F9C0F9E01015C
:100E7000000E5E6F600E5F6F3D0E606F080E616F5B
:100E8000010147BF50EF07F0486750EF07F049678F
:100E900050EF07F04A6750EF07F0F28875EF07F060
:100EA000F2985E6B5F6B606B616B966B976B986B88
:100EB000996B9A6B9B6B9C6B9D6B9E6B9F6BA06BF6
:100EC000A16BA26BA36BA46BA56BA66BA76BA86BA6
:100ED000A96BAA6BAB6BAC6BAD6BAE6BAF6BB06B56
:100EE000B16BB26BB36BB46BB56BD76AD66A0101E9
:100EF000456B466B0CC100F10DC101F10EC102F151
:100F00000FC103F110C104F111C105F112C106F1C5
:100F100013C107F114C108F115C109F116C10AF195
:100F200017C10BF135C134F196EF07F002C0E0FFB5
:100F3000005001C0D8FF1000A6B29CEF07F00CC013
:100F4000A9FF0BC0A8FFA69EA69CA684F29E550EE4
:100F5000A76EAA0EA76EA682F28EA694A6B2AEEFD8
:100F600007F00C2A1200A96EA69EA69CA680A85087
:100F70000C2A120004012C0E826FCCEC0AF05AEC01
:100F800020F00C50B3EC07F0E8CF00F10C50B3ECBC
:100F900007F0E8CF01F101AFD3EF07F00101FF0E39
:100FA000026FFF0E036FFDEC1FF02967DFEF07F004
:100FB0000401200E826FCCEC0AF0E4EF07F004018C
:100FC0002D0E826FCCEC0AF027EC1EF01200076A9F
:100FD0000F6A106A0F010D0EC16E860EC06E030EF1
:100FE000C26E0F01680E896E130E926E080E8A6E25
:100FF000F30E936E8B6A900E946EF18EF19E0E6AD4
:1010000001015B6B5C6B5D6B576B586BF29A010176
:10101000476B486B496B4A6B4B6B4C6B4D6B4E6B24
:101020004F6B506B516B526B456B466BD76AD66AF0
:101030000F01280ED56EF28A9D90B00ECD6E010183
:101040005E6B5F6B606B616B626B636B646B656B3C
:10105000666B676B686B696B536B546BCF6ACE6A58
:101060000F9A0F9C0F9E9D80760ECA6E9D82020184
:101070003C0E006FCC6A160EB3EC07F0E8CF00F11F
:10108000170EB3EC07F0E8CF01F1180EB3EC07F040
:10109000E8CF02F1190EB3EC07F0E8CF03F101013C
:1010A00003AF6DEF08F05AEC20F0160E0C6E00C185
:1010B0000BF09CEC07F0170E0C6E01C10BF09CECD2
:1010C00007F0180E0C6E02C10BF09CEC07F0190E25
:1010D0000C6E03C10BF09CEC07F000C18AF101C15A
:1010E0008BF102C18CF103C18DF100C18EF101C100
:1010F0008FF102C190F103C191F11A0EB3EC07F028
:10110000E8CF00F11B0EB3EC07F0E8CF01F11C0EA5
:10111000B3EC07F0E8CF02F11D0EB3EC07F0E8CF17
:1011200003F1010103AFC3EF08F05AEC20F01A0EEF
:101130000C6E00C10BF09CEC07F01B0E0C6E01C195
:101140000BF09CEC07F01C0E0C6E02C10BF09CEC3B
:1011500007F01D0E0C6E03C10BF09CEC07F01A0E8D
:10116000B3EC07F0E8CF00F11B0EB3EC07F0E8CFCB
:1011700001F11C0EB3EC07F0E8CF02F11D0EB3EC49
:1011800007F0E8CF03F100C192F101C193F102C170
:1011900094F103C195F1240EAC6E900EAB6E240E4B
:1011A000AC6E080EB86E000EB06E1F0EAF6E04016E
:1011B000806B816B0F01900EAB6E0F019D8A030156
:1011C000806B816BC26B8B92BCEC26F06DEC29F0CE
:1011D0009CEC24F0200EB3EC07F0E8CF2FF50501CE
:1011E0002F51FF0AD8A4FCEF08F02F6B200E0C6ED5
:1011F0002FC50BF09CEC07F00501010E306F3C0E83
:10120000316F250EB3EC07F0E8CF00F1260EB3ECFA
:1012100007F0E8CF01F1270EB3EC07F0E8CF02F1B9
:10122000280EB3EC07F0E8CF03F1010103AF33EF71
:1012300009F05AEC20F0250E0C6E00C10BF09CEC6E
:1012400007F0260E0C6E01C10BF09CEC07F0270E88
:101250000C6E02C10BF09CEC07F0280E0C6E03C163
:101260000BF09CEC07F000C153F501C154F502C12D
:1012700055F503C156F500C157F501C158F502C136
:1012800059F503C15AF5290EB3EC07F0E8CF5BF529
:1012900005015C515B5DD8A05BC55CF505012F5174
:1012A000020A0EE181B860EF09F005015C2F5DEFE5
:1012B00009F05BC55CF560EF09F081BAACEF29F08D
:1012C000210EB3EC07F0E8CF00F1220EB3EC07F0EB
:1012D000E8CF01F1230EB3EC07F0E8CF02F1240EC2
:1012E000B3EC07F0E8CF03F1010103AFA6EF09F07B
:1012F0005AEC20F0210E0C6E00C10BF09CEC07F0B4
:10130000220E0C6E01C10BF09CEC07F0230E0C6E4C
:1013100002C10BF09CEC07F0240E0C6E03C10BF025
:101320009CEC07F0210EB3EC07F0E8CF00F1220EA1
:10133000B3EC07F0E8CF01F1230EB3EC07F0E8CFF0
:1013400002F1240EB3EC07F0E8CF03F100C15DF524
:1013500001C15EF502C15FF503C160F5D3EC23F076
:1013600095EC22F0E5EC21F005012F51030A12E083
:1013700005012F51040A1DE005012F51050A24E043
:1013800005012F51060A32E005012F51070A38E006
:1013900009EF0AF0ACC500F101010F0E00170101C1
:1013A0000051000A36E001010051050A32E006EF63
:1013B0000AF0ACC500F101010F0E00170101005148
:1013C000000A27E006EF0AF00501AC51000A21E00F
:1013D0000501AC51150A1DE00501AC51300A19E0B8
:1013E0000501AC51450A15E006EF0AF00501AC51C4
:1013F000000A0FE00501AC51300A0BE006EF0AF0DD
:101400000501AC51000A05E006EF0AF081BAACEF25
:1014100029F00F94C8EC20F08A840501006B016B61
:10142000026B036B046B056B066B0D6B0E6B0F6B26
:10143000106B116B126B196B1A6B1B6B1C6B1D6B9A
:101440001E6B1F6B206B136B146B156B166B176B7E
:10145000186B0501626B636B07900001F28EF28CD2
:1014600007B0A6EF1CF00FB087EF17F00FB89FEF93
:1014700010F00301805181197F0BD8B4A6EF1CF046
:1014800013EE00F081517F0BE126812BE7CFE8FFBF
:10149000E00BD8B4A6EF1CF023EE82F0C2513F0B54
:1014A000D926E7CFDFFFC22BDF50780AD8A4A6EFFA
:1014B0001CF007808EC100F18FC101F190C102F1D3
:1014C00091C103F10101040E046F000E056F000EBF
:1014D000066F000E076F5FEC1FF000AF79EF0AF0A8
:1014E0000101030E8E6F000E8F6F000E906F000EC5
:1014F000916F03018251720AD8B487EF17F08251BD
:10150000520AD8B487EF17F08251750AD8B487EF22
:1015100017F08251630AD8B462EF19F08251690A58
:10152000D8B442EF14F082517A0AD8B455EF15F0CE
:101530008251490AD8B4E1EF13F08251500AD8B46D
:10154000FFEF12F08251700AD8B442EF13F08251CB
:10155000540AD8B46DEF13F08251740AD8B4B3EFC3
:1015600013F08251730AD8B4B7EF16F08251530AC0
:10157000D8B41CEF17F082514C0AD8B4E0EF0AF04F
:101580008251470AD8B453EF12F08251670AD8B497
:101590007BEF12F097EF19F0040114EE00F0805188
:1015A0007F0BE12682C4E7FF802B120004010D0EA1
:1015B000826FCCEC0AF00A0E826FCCEC0AF01200BB
:1015C00003018351300AD8B4A1EF0DF00301835118
:1015D000310AD8B4ADEF0EF003018351320AD8B40A
:1015E00019EF0FF003018351330AD8B427EF0FF03E
:1015F00003018351340AD8B435EF0FF0030183514E
:10160000350AD8B4A4EF10F003018351360AD8B4D8
:10161000D2EF10F003018351460AD8B4F8EF0FF06F
:10162000030183514D0AD8B41AEF0CF00301835122
:101630006D0AD8B434EF0CF0030183515A0AD8B4C0
:1016400027EF0EF003018351490AD8B4D2EF11F00D
:1016500003018351500AD8B404EF11F00301835100
:10166000540AD8B47DEF11F003018351630AD8B452
:1016700054EF0CF003018351430AD8B44CEF0DF042
:1016800003018351730AD8B452EF0CF00301835164
:10169000610AD8B467EF0BF003018351650AD8B42F
:1016A000EFEF0DF003018351450AD8B4FDEF0DF0C3
:1016B00003018351620AD8B40BEF0EF0030183518A
:1016C000420AD8B419EF0EF0D8A497EF19F004012C
:1016D0004C0E826FCCEC0AF00401610E826FCCECF0
:1016E0000AF095EC22F004012C0E826FCCEC0AF08B
:1016F0005AEC20F0ABC500F10101FDEC1FF031C147
:1017000082F40401300E8227CCEC0AF032C182F45C
:101710000401300E8227CCEC0AF033C182F40401BC
:10172000300E8227CCEC0AF004012C0E826FCCEC38
:101730000AF05AEC20F0ACC500F10101FDEC1FF0FD
:1017400031C182F40401300E8227CCEC0AF032C1A0
:1017500082F40401300E8227CCEC0AF033C182F40B
:101760000401300E8227CCEC0AF004012C0E826FAB
:10177000CCEC0AF05AEC20F0ADC500F10101FDEC13
:101780001FF031C182F40401300E8227CCEC0AF044
:1017900032C182F40401300E8227CCEC0AF033C14E
:1017A00082F40401300E8227CCEC0AF004012C0EE6
:1017B000826FCCEC0AF05AEC20F0AEC500F10101CA
:1017C000FDEC1FF031C182F40401300E8227CCEC15
:1017D0000AF032C182F40401300E8227CCEC0AF008
:1017E00033C182F40401300E8227CCEC0AF00401EC
:1017F0002C0E826FCCEC0AF05AEC20F0B3C500F14D
:101800000101FDEC1FF031C182F40401300E82278A
:10181000CCEC0AF032C182F40401300E8227CCEC09
:101820000AF033C182F40401300E8227CCEC0AF0B6
:1018300000EF11F09BEC20F084C333F1A8EC20F012
:101840001FEC20F0200E0C6E00C10BF09CEC07F09A
:1018500000C12FF505012F51000A06E005012F51A7
:10186000010A02E03BEC23F004014C0E826FCCEC49
:101870000AF004014D0E826FCCEC0AF004012C0E2C
:10188000826FCCEC0AF05AEC20F02FC500F1FDEC91
:101890001FF033C182F40401300E8227CCEC0AF031
:1018A00000EF11F0ACEF29F004014C0E826FCCEC8C
:1018B0000AF00401630E826FCCEC0AF0E5EC21F033
:1018C00004012C0E826FCCEC0AF069EC0CF000EFF6
:1018D00011F05AEC20F0B1C500F10101003B0F0EF0
:1018E0000017FDEC1FF033C182F40401300E822793
:1018F000CCEC0AF0B1C500F101010F0E0101001797
:10190000FDEC1FF033C182F40401300E8227CCECD1
:101910000AF004012D0E826FCCEC0AF0B0C500F184
:101920000101003B0F0E0017FDEC1FF033C182F4E4
:101930000401300E8227CCEC0AF0B0C500F10101A1
:101940000F0E01010017FDEC1FF033C182F40401FA
:10195000300E8227CCEC0AF004012D0E826FCCEC05
:101960000AF0AFC500F10101003B0F0E0017FDECBE
:101970001FF033C182F40401300E8227CCEC0AF050
:10198000AFC500F101010F0E01010017FDEC1FF0C2
:1019900033C182F40401300E8227CCEC0AF004013A
:1019A000200E826FCCEC0AF0AEC500F10F0E0101E3
:1019B0000017FDEC1FF033C182F40401300E8227C2
:1019C000CCEC0AF00401200E826FCCEC0AF0ADC51D
:1019D00000F101010101003B0F0E0017FDEC1FF0AB
:1019E00033C182F40401300E8227CCEC0AF0ADC57D
:1019F00000F101010F0E01010017FDEC1FF033C1D2
:101A000082F40401300E8227CCEC0AF004013A0E75
:101A1000826FCCEC0AF0ACC500F10101003B0F0E67
:101A20000017FDEC1FF033C182F40401300E822751
:101A3000CCEC0AF0ACC500F101010F0E010100175A
:101A4000FDEC1FF033C182F40401300E8227CCEC90
:101A50000AF004013A0E826FCCEC0AF0ABC500F13B
:101A60000101003B0F0E0017FDEC1FF033C182F4A3
:101A70000401300E8227CCEC0AF0ABC500F1010165
:101A80000F0E0017FDEC1FF033C182F40401300E7D
:101A90008227CCEC0AF0120084C3E8FF0F0BE83A6F
:101AA000E8CFB1F585C3E8FF0F0B0501B11387C37C
:101AB000E8FF0F0BE83AE8CFB0F588C3E8FF0F0B5B
:101AC0000501B0138AC3E8FF0F0BE83AE8CFAFF582
:101AD0008BC3E8FF0F0B0501AF138DC3E8FF0F0B9E
:101AE000E8CFAEF58FC3E8FF0F0BE83AE8CFADF5CE
:101AF00090C3E8FF0F0B0501AD1392C3E8FF0F0B76
:101B0000E83AE8CFACF593C3E8FF0F0B0501AC133F
:101B100095C3E8FF0F0BE83AE8CFABF596C3E8FFB3
:101B20000F0B0501AB1344EC22F004014C0E826F45
:101B3000CCEC0AF00401430E826FCCEC0AF05EEFAD
:101B40000CF06DEC29F05AEC20F02DC500F1FDEC05
:101B50001FF004014C0E826FCCEC0AF00401300E31
:101B6000826FCCEC0AF004012C0E826FCCEC0AF0F0
:101B700031C182F40401300E8227CCEC0AF032C16C
:101B800082F40401300E8227CCEC0AF033C182F4D7
:101B90000401300E8227CCEC0AF004012C0E826F77
:101BA000CCEC0AF05AEC20F02EC500F1FDEC1FF051
:101BB00031C182F40401300E8227CCEC0AF032C12C
:101BC00082F40401300E8227CCEC0AF033C182F497
:101BD0000401300E8227CCEC0AF000EF11F0040172
:101BE0004C0E826FCCEC0AF00401650E826FCCECD7
:101BF0000AF024EC24F000EF11F004014C0E826F87
:101C0000CCEC0AF00401450E826FCCEC0AF041ECFA
:101C100024F000EF11F004014C0E826FCCEC0AF0BE
:101C20000401620E826FCCEC0AF07BEC24F000EF32
:101C300011F004014C0E826FCCEC0AF00401420E4C
:101C4000826FCCEC0AF05EEC24F000EF11F004019E
:101C50004C0E826FCCEC0AF004015A0E826FCCEC71
:101C60000AF004012C0E826FCCEC0AF06DEC29F026
:101C70005AEC20F005012E51130A06E005012E5101
:101C8000170A0DE058EF0EF00101000E006F000E74
:101C9000016F100E026F000E036F58EF0EF001017E
:101CA000000E006F000E016F000E026F010E036F39
:101CB0000101100E046F000E056F000E066F000E7E
:101CC000076F90EC1FF0FDEC1FF02AC182F40401B5
:101CD000300E8227CCEC0AF02BC182F40401300EC6
:101CE0008227CCEC0AF02CC182F40401300E82274A
:101CF000CCEC0AF02DC182F40401300E8227CCEC2A
:101D00000AF02EC182F40401300E8227CCEC0AF0D6
:101D10002FC182F40401300E8227CCEC0AF030C1CE
:101D200082F40401300E8227CCEC0AF031C182F437
:101D30000401300E8227CCEC0AF032C182F4040197
:101D4000300E8227CCEC0AF033C182F40401300E4D
:101D50008227CCEC0AF000EF11F004014C0E826FE8
:101D6000CCEC0AF00401310E826FCCEC0AF00401D5
:101D70002C0E826FCCEC0AF025C500F126C501F1CE
:101D800027C502F128C503F10101100E046F000EF2
:101D9000056F000E066F000E076F90EC1FF0FDEC54
:101DA0001FF02AC182F40401300E8227CCEC0AF025
:101DB0002BC182F40401300E8227CCEC0AF02CC136
:101DC00082F40401300E8227CCEC0AF02DC182F49B
:101DD0000401300E8227CCEC0AF02EC182F40401FB
:101DE000300E8227CCEC0AF02FC182F40401300EB1
:101DF0008227CCEC0AF030C182F40401300E822735
:101E0000CCEC0AF031C182F40401300E8227CCEC14
:101E10000AF032C182F40401300E8227CCEC0AF0C1
:101E200033C182F40401300E8227CCEC0AF000EFBB
:101E300011F004014C0E826FCCEC0AF00401320E5A
:101E4000826FCCEC0AF072EC26F000EF11F0040186
:101E50004C0E826FCCEC0AF00401330E826FCCEC96
:101E60000AF0CFEC26F0B7EF0EF004014C0E826FB3
:101E7000CCEC0AF00401340E826FCCEC0AF00401C1
:101E80002C0E826FCCEC0AF09BEC20F084C32AF17C
:101E900085C32BF186C32CF187C32DF188C32EF1A6
:101EA00089C32FF18AC330F18BC331F18CC332F176
:101EB0008DC333F10101296BA8EC20F01FEC20F059
:101EC000100E046F000E056F000E066F000E076FF8
:101ED00070EC1FF000C121F501C122F502C123F50C
:101EE00003C124F520EC29F034C5ABF535C5ACF5BC
:101EF00036C5ADF537C5AEF538C5AFF539C5B0F562
:101F00003AC5B1F569EC0CF004012C0E826FCCECF3
:101F10000AF03BC500F13CC501F13DC502F13EC5EB
:101F200003F10101000E046F000E056F010E066F34
:101F3000000E076F90EC1FF0FDEC1FF02967A3EF78
:101F40000FF0A8EF0FF004012D0E826FCCEC0AF019
:101F500030C182F40401300E8227CCEC0AF031C18A
:101F600082F40401300E8227CCEC0AF004012E0E1C
:101F7000826FCCEC0AF032C182F40401300E822769
:101F8000CCEC0AF033C182F40401300E8227CCEC91
:101F90000AF004012C0E826FCCEC0AF05AEC20F00F
:101FA0003FC500F140C501F1C1EC1AF004012C0E4F
:101FB000826FCCEC0AF05AEC20F041C500F1FDEC48
:101FC0001FF031C182F40401300E8227CCEC0AF0FC
:101FD00032C182F40401300E8227CCEC0AF033C106
:101FE00082F40401300E8227CCEC0AF000EF11F0ED
:101FF0009BEC20F085C32AF186C32BF187C32CF11B
:1020000088C32DF189C32EF18AC32FF18BC330F120
:102010008CC331F18DC332F18EC333F10101296BD1
:10202000A8EC20F01FEC20F00101010E046F000E5F
:10203000056F000E066F000E076F5FEC1FF0100EAD
:10204000046F000E056F000E066F000E076F70EC38
:102050001FF000C129F501C12AF502C12BF503C10A
:102060002CF5FBEC25F004014C0E826FCCEC0AF051
:102070000401460E826FCCEC0AF004012C0E826F34
:10208000CCEC0AF025C500F126C501F127C502F107
:1020900028C503F10101100E046F000E056F000E3C
:1020A000066F000E076F90EC1FF0FDEC1FF02AC1C9
:1020B00082F40401300E8227CCEC0AF02BC182F4AA
:1020C0000401300E8227CCEC0AF02CC182F404010A
:1020D000300E8227CCEC0AF02DC182F40401300EC0
:1020E0008227CCEC0AF02EC182F40401300E822744
:1020F000CCEC0AF02FC182F40401300E8227CCEC24
:102100000AF030C182F40401300E8227CCEC0AF0D0
:1021100031C182F40401300E8227CCEC0AF032C1C6
:1021200082F40401300E8227CCEC0AF033C182F431
:102130000401300E8227CCEC0AF000EF11F00F986A
:10214000CFEC26F000EF11F004014C0E826FCCECC6
:102150000AF00401350E826FCCEC0AF004012C0E5B
:10216000826FCCEC0AF05AEC20F00784B5C500F180
:102170000794FDEC1FF031C182F40401300E822778
:10218000CCEC0AF032C182F40401300E8227CCEC90
:102190000AF033C182F40401300E8227CCEC0AF03D
:1021A00000EF11F092EC26F05AEC20F033C500F16C
:1021B000FDEC1FF004014C0E826FCCEC0AF0040120
:1021C000360E826FCCEC0AF004012C0E826FCCEC40
:1021D0000AF031C182F40401300E8227CCEC0AF0FF
:1021E00032C182F40401300E8227CCEC0AF033C1F4
:1021F00082F40401300E8227CCEC0AF000EF11F0DB
:10220000D6EC0AF097EF19F004014C0E826FCCEC7B
:102210000AF00401500E826FCCEC0AF004012C0E7F
:10222000826FCCEC0AF085C32AF186C32BF187C3F9
:102230002CF188C32DF189C32EF18AC32FF18BC3F2
:1022400030F18CC331F18DC332F18EC333F1010112
:10225000A8EC20F01FEC20F003018451530A0DE09C
:10226000030184514D0A38E00401780E826FCCECF2
:102270000AF0D6EC0AF097EF19F00401530E826FC2
:10228000CCEC0AF0250E0C6E00C10BF09CEC07F0B4
:10229000260E0C6E01C10BF09CEC07F0270E0C6EA5
:1022A00002C10BF09CEC07F0280E0C6E03C10BF082
:1022B0009CEC07F000C153F501C154F502C155F57E
:1022C00003C156F500C157F501C158F502C159F5D2
:1022D00003C15AF5E1EF11F004014D0E826FCCEC11
:1022E0000AF0290E0C6E00C10BF09CEC07F000C147
:1022F0005BF500C15CF5E1EF11F004014C0E826F5B
:10230000CCEC0AF00401540E826FCCEC0AF004010C
:102310002C0E826FCCEC0AF084C32AF185C32BF11A
:1023200086C32CF187C32DF188C32EF189C32FF109
:102330008AC330F18BC331F18DC332F18EC333F1D7
:102340000101A8EC20F01FEC20F00101000E046F49
:10235000000E056F010E066F000E076F70EC1FF088
:10236000210E0C6E00C10BF09CEC07F0220E0C6EDF
:1023700001C10BF09CEC07F0230E0C6E02C10BF0B8
:102380009CEC07F0240E0C6E03C10BF09CEC07F0E4
:1023900000C15DF501C15EF502C15FF503C160F5E5
:1023A000E1EF11F004014C0E826FCCEC0AF0040155
:1023B000490E826FCCEC0AF004012C0E826FCCEC3B
:1023C0000AF0250EB3EC07F0E8CF00F1260EB3ECCF
:1023D00007F0E8CF01F1270EB3EC07F0E8CF02F1E8
:1023E000280EB3EC07F0E8CF03F1FDEC1FF0E0ECB2
:1023F0001DF00401730E826FCCEC0AF004012C0E68
:10240000826FCCEC0AF05AEC20F0290EB3EC07F006
:10241000E8CF00F1FDEC1FF0E0EC1DF00401730EBD
:10242000826FCCEC0AF004012C0E826FCCEC0AF027
:1024300057C500F158C501F159C502F15AC503F15C
:10244000FDEC1FF0E0EC1DF00401730E826FCCEC8C
:102450000AF004012C0E826FCCEC0AF05AEC20F04A
:102460005CC500F1FDEC1FF0E0EC1DF004016D0E09
:10247000826FCCEC0AF004012C0E826FCCEC0AF0D7
:102480005DC500F15EC501F15FC502F160C503F1F4
:10249000B2EC19F004012C0E826FCCEC0AF0D6ECF1
:1024A0000AF097EF19F023EE82F0010EC26FC251CD
:1024B000D926DFCFC3F3C22B780EC319D8B465EF8A
:1024C00012F0DCEC20F057EF12F00D0EC36FDCECD5
:1024D00020F00A0EC36FDCEC20F00401670E826F5F
:1024E000CCEC0AF00401420E826FCCEC0AF0D6EC80
:1024F0000AF097EF19F003018351300A27E0030136
:102500008351310A29E003018351320A2BE0030190
:102510008351340A2DE003018351350A2FE0030172
:102520008351360A31E003018351380A33E0030155
:102530008351410A35E003018351420A37E0030128
:102540008351430A39E0D8A497EF19F00DC502F57D
:102550000EC503F5E2EF12F00FC502F510C503F545
:10256000E2EF12F011C502F512C503F5E2EF12F029
:1025700019C502F51AC503F5E2EF12F01BC502F505
:102580001CC503F5E2EF12F01DC502F51EC503F5EB
:10259000E2EF12F01FC502F520C503F5E2EF12F0DD
:1025A00013C502F514C503F5E2EF12F015C502F5E7
:1025B00016C503F5E2EF12F017C502F518C503F5CD
:1025C000E2EF12F027EE00F005010251D926035187
:1025D000D8B00329DA26DFCFE8FF0A0A0CE0DFCF04
:1025E00082F4CCEC0AF00501032B023F0307030E33
:1025F0000317E2EF12F0D6EC0AF097EF19F083C35D
:102600002AF184C32BF185C32CF186C32DF187C336
:102610002EF188C32FF189C330F18AC331F18BC306
:1026200032F18CC333F10101A8EC20F01FEC20F053
:10263000160E0C6E00C10BF09CEC07F0170E0C6E22
:1026400001C10BF09CEC07F0180E0C6E02C10BF0F0
:102650009CEC07F0190E0C6E03C10BF09CEC07F01C
:1026600000C18AF101C18BF102C18CF103C18DF16E
:1026700000C18EF101C18FF102C190F103C191F14E
:10268000E1EF13F083C32AF184C32BF185C32CF14E
:1026900086C32DF187C32EF188C32FF189C330F192
:1026A0008AC331F18BC332F18CC333F10101A8EC41
:1026B00020F01FEC20F000C18AF101C18BF102C1B2
:1026C0008CF103C18DF100C18EF101C18FF102C106
:1026D00090F103C191F1E1EF13F083C32AF184C3B8
:1026E0002BF185C32CF186C32DF187C32EF188C34E
:1026F0002FF189C330F18AC331F18CC332F18DC31C
:1027000033F10101A8EC20F01FEC20F00101000ED4
:10271000046F000E056F010E066F000E076F70EC60
:102720001FF01A0E0C6E00C10BF09CEC07F01B0E94
:102730000C6E01C10BF09CEC07F01C0E0C6E02C17C
:102740000BF09CEC07F01D0E0C6E03C10BF09CEC23
:1027500007F000C192F101C193F102C194F103C1EC
:1027600095F1E1EF13F083C32AF184C32BF185C304
:102770002CF186C32DF187C32EF188C32FF189C3B5
:1027800030F18AC331F18CC332F18DC333F10101D1
:10279000A8EC20F01FEC20F00101000E046F000EE9
:1027A000056F010E066F000E076F70EC1FF000C181
:1027B00092F101C193F102C194F103C195F1E1EFEE
:1027C00013F0160EB3EC07F0E8CF00F1170EB3ECE0
:1027D00007F0E8CF01F1180EB3EC07F0E8CF02F1F3
:1027E000190EB3EC07F0E8CF03F1FDEC1FF0E0ECBD
:1027F0001DF00401730E826FCCEC0AF004012C0E64
:10280000826FCCEC0AF08AC100F18BC101F18CC15E
:1028100002F18DC103F1FDEC1FF0E0EC1DF00401AD
:10282000730E826FCCEC0AF004012C0E826FCCEC9C
:102830000AF01A0EB3EC07F0E8CF00F11B0EB3EC70
:1028400007F0E8CF01F11C0EB3EC07F0E8CF02F17E
:102850001D0EB3EC07F0E8CF03F1B2EC19F0040160
:102860002C0E826FCCEC0AF092C100F193C101F101
:1028700094C102F195C103F1B2EC19F0D6EC0AF063
:1028800097EF19F00401690E826FCCEC0AF0040195
:102890002C0E826FCCEC0AF00101040E006F000ECA
:1028A000016F000E026F000E036FFDEC1FF02CC1D4
:1028B00082F40401300E8227CCEC0AF02DC182F4A0
:1028C0000401300E8227CCEC0AF02EC182F4040100
:1028D000300E8227CCEC0AF02FC182F40401300EB6
:1028E0008227CCEC0AF030C182F40401300E82273A
:1028F000CCEC0AF031C182F40401300E8227CCEC1A
:102900000AF032C182F40401300E8227CCEC0AF0C6
:1029100033C182F40401300E8227CCEC0AF00401AA
:102920002C0E826FCCEC0AF00101070E006F000E36
:10293000016F000E026F000E036FFDEC1FF02CC143
:1029400082F40401300E8227CCEC0AF02DC182F40F
:102950000401300E8227CCEC0AF02EC182F404016F
:10296000300E8227CCEC0AF02FC182F40401300E25
:102970008227CCEC0AF030C182F40401300E8227A9
:10298000CCEC0AF031C182F40401300E8227CCEC89
:102990000AF032C182F40401300E8227CCEC0AF036
:1029A00033C182F40401300E8227CCEC0AF004011A
:1029B0002C0E826FCCEC0AF001011C0E006F000E91
:1029C000016F000E026F000E036FFDEC1FF02CC1B3
:1029D00082F40401300E8227CCEC0AF02DC182F47F
:1029E0000401300E8227CCEC0AF02EC182F40401DF
:1029F000300E8227CCEC0AF02FC182F40401300E95
:102A00008227CCEC0AF030C182F40401300E822718
:102A1000CCEC0AF031C182F40401300E8227CCECF8
:102A20000AF032C182F40401300E8227CCEC0AF0A5
:102A300033C182F40401300E8227CCEC0AF0040189
:102A40002C0E826FCCEC0AF0200EF86EF76AF66A54
:102A500004010900F5CF82F4CCEC0AF00900F5CFAF
:102A600082F4CCEC0AF00900F5CF82F4CCEC0AF049
:102A70000900F5CF82F4CCEC0AF00900F5CF82F41E
:102A8000CCEC0AF00900F5CF82F4CCEC0AF0090096
:102A9000F5CF82F4CCEC0AF00900F5CF82F4CCEC4F
:102AA0000AF0D6EC0AF097EF19F08351630AD8A424
:102AB00097EF19F08451610AD8A497EF19F0855166
:102AC0006C0AD8A497EF19F08651410A42E086516A
:102AD000440A1BE08651420AD8B4BCEF15F0865177
:102AE000350AD8B421EF1BF08651360AD8B476EFF8
:102AF0001BF08651370AD8B4DFEF1BF08651380A35
:102B0000D8B43DEF1CF097EF19F00798079A04012D
:102B10007A0E826FCCEC0AF00401780E826FCCEC56
:102B20000AF00401640E826FCCEC0AF081A8A0EFD9
:102B300015F00401550E826FCCEC0AF0A5EF15F0EC
:102B400004014C0E826FCCEC0AF0D6EC0AF097EF41
:102B500019F00788079A04017A0E826FCCEC0AF00C
:102B60000401410E826FCCEC0AF00401610E826F09
:102B7000CCEC0AF096EF15F00798078A04017A0E5C
:102B8000826FCCEC0AF00401420E826FCCEC0AF0AA
:102B90000401610E826FCCEC0AF096EF15F0010192
:102BA0006667DAEF15F06767DAEF15F06867DAEF56
:102BB00015F06967F2EF15F04F67E6EF15F0506713
:102BC000E6EF15F05167E6EF15F05267F2EF15F0FA
:102BD0000101000E006F000E016F000E026F000E6B
:102BE000036F12000101620E046F010E056F000EEB
:102BF000066F000E076F66C100F167C101F168C181
:102C000002F169C103F15FEC1FF003BF76EF16F02C
:102C10000101000E046FA80E056F550E066F020E1F
:102C2000076F66C100F167C101F168C102F169C1B6
:102C300003F166C186F167C187F168C188F169C196
:102C400089F15FEC1FF003BF2FEF16F00101000EBA
:102C5000866FA80E876F550E886F020E896F0E0E55
:102C6000B3EC07F0E8CF18F10F0EB3EC07F0E8CFA4
:102C700019F1100EB3EC07F0E8CF1AF1110EB3EC16
:102C800007F0E8CF1BF1A8EC1EF086C104F187C164
:102C900005F188C106F189C107F15FEC1FF00782D9
:102CA0006CEC1EF0A8EC1EF007926CEC1EF086C1D6
:102CB00000F187C101F188C102F189C103F10792D6
:102CC0006CEC1EF0CC0E046FE00E056F870E066FE5
:102CD000050E076F5FEC1FF000C118F101C119F17B
:102CE00002C11AF103C11BF1AEEF16F00101800E13
:102CF000006F1A0E016F060E026F000E036F4FC1B8
:102D000004F150C105F151C106F152C107F15FEC68
:102D10001FF003AF8FEF16F05AEC20F012000E0EEA
:102D2000B3EC07F0E8CF18F10F0EB3EC07F0E8CFE3
:102D300019F1100EB3EC07F0E8CF1AF1110EB3EC55
:102D400007F0E8CF1BF14FC100F150C101F151C1B3
:102D500002F152C103F107826CEC1EF018C100F1C0
:102D600019C101F11AC102F11BC103F112000401E2
:102D7000730E826FCCEC0AF004012C0E826FCCEC47
:102D80000AF0078462C166F163C167F164C168F14A
:102D900065C169F14BC14FF14CC150F14DC151F1C9
:102DA0004EC152F157C159F158C15AF10794DDECA7
:102DB00016F0D6EC0AF097EF19F066C100F167C182
:102DC00001F168C102F169C103F10101FDEC1FF0DD
:102DD000E0EC1DF00401630E826FCCEC0AF00401FC
:102DE0002C0E826FCCEC0AF04FC100F150C101F102
:102DF00051C102F152C103F10101FDEC1FF0E0EC01
:102E00001DF00401660E826FCCEC0AF004012C0E5A
:102E1000826FCCEC0AF05AEC20F059C100F15AC193
:102E200001F10101FDEC1FF0E0EC1DF00401740E56
:102E3000826FCCEC0AF0120010820401530E826FF4
:102E4000CCEC0AF004012C0E826FCCEC0AF083C3A8
:102E50002AF184C32BF185C32CF186C32DF187C3DE
:102E60002EF188C32FF189C330F18AC331F18BC3AE
:102E700032F18CC333F10101A8EC20F01FEC20F0FB
:102E800000C166F101C167F102C168F103C169F1D6
:102E90008EC32AF18FC32BF190C32CF191C32DF176
:102EA00092C32EF193C32FF194C330F195C331F146
:102EB00096C332F197C333F10101A8EC20F01FEC67
:102EC00020F000C14FF101C150F102C151F103C125
:102ED00052F19BEC20F099C32FF19AC330F19BC3C0
:102EE00031F19CC332F19DC333F10101A8EC20F014
:102EF0001FEC20F000C159F101C15AF1DDEC16F0D0
:102F000004012C0E826FCCEC0AF08EEF17F0825188
:102F1000520A03E10F828EEF17F00F928251750A69
:102F200003E1108495EF17F010948251550A03E1E4
:102F300010869CEF17F01096078410B2F9EF17F087
:102F400010A4E5EF17F0B6C166F1B7C167F1B8C1DB
:102F500068F1B9C169F1BAC16AF1BBC16BF1BCC119
:102F60006CF1BDC16DF1BEC16EF1BFC16FF1C0C1E9
:102F700070F1C1C171F1C2C172F1C3C173F1C4C1B9
:102F800074F1C5C175F1C6C176F1C7C177F1C8C189
:102F900078F1C9C179F1CAC17AF1CBC17BF1CCC159
:102FA0007CF1CDC17DF1CEC17EF1CFC17FF1D0C129
:102FB00080F1D1C181F1D2C182F1D3C183F1D4C1F9
:102FC00084F1D5C185F1EDEF17F062C166F163C1FF
:102FD00067F164C168F165C169F14BC14FF14CC142
:102FE00050F14DC151F14EC152F157C159F158C183
:102FF0005AF107940FA01BEF18F00101926708EF38
:1030000018F0936708EF18F0946708EF18F09567C9
:103010000CEF18F01BEF18F0CFEC15F092C104F193
:1030200093C105F194C106F195C107F15FEC1FF062
:1030300003BF5FEF19F0CFEC15F00101000E046F34
:10304000000E056F010E066F000E076F90EC1FF06B
:1030500010A432EF18F00401750E826FCCEC0AF068
:1030600037EF18F00401720E826FCCEC0AF0040105
:103070002C0E826FCCEC0AF0FDEC1FF0296746EFB6
:1030800018F00401200E826F49EF18F004012D0E94
:10309000826FCCEC0AF030C182F40401300E82273A
:1030A000CCEC0AF031C182F40401300E8227CCEC62
:1030B0000AF004012E0E826FCCEC0AF032C182F4C9
:1030C0000401300E8227CCEC0AF033C182F40401F3
:1030D000300E8227CCEC0AF004016D0E826FCCEC2E
:1030E0000AF004012C0E826FCCEC0AF04FC100F103
:1030F00050C101F151C102F152C103F10101FDECD6
:103100001FF0E0EC1DF00401480E826FCCEC0AF0D9
:1031100004017A0E826FCCEC0AF004012C0E826F4F
:10312000CCEC0AF066C100F167C101F168C102F19F
:1031300069C103F10101FDEC1FF0E0EC1DF0040199
:10314000630E826FCCEC0AF004012C0E826FCCEC83
:103150000AF066C100F167C101F168C102F169C1FD
:1031600003F101010A0E046F000E056F000E066FD9
:10317000000E076F70EC1FF0000E046F120E056F4B
:10318000000E066F000E076F90EC1FF0FDEC1FF0B5
:103190002AC182F40401300E8227CCEC0AF02BC144
:1031A00082F40401300E8227CCEC0AF02CC182F4A8
:1031B0000401300E8227CCEC0AF02DC182F4040108
:1031C000300E8227CCEC0AF02EC182F40401300EBE
:1031D0008227CCEC0AF02FC182F40401300E822742
:1031E000CCEC0AF030C182F40401300E8227CCEC22
:1031F0000AF004012E0E826FCCEC0AF031C182F489
:103200000401300E8227CCEC0AF032C182F40401B2
:10321000300E8227CCEC0AF033C182F40401300E68
:103220008227CCEC0AF00401730E826FCCEC0AF01A
:1032300004012C0E826FCCEC0AF05AEC20F059C13C
:1032400000F15AC101F1C1EC1AF00FB22BEF19F0E5
:103250000FA05DEF19F004012C0E826FCCEC0AF088
:10326000200EF86EF76AF66A04010900F5CF82F4C1
:10327000CCEC0AF00900F5CF82F4CCEC0AF009009E
:10328000F5CF82F4CCEC0AF00900F5CF82F4CCEC57
:103290000AF00900F5CF82F4CCEC0AF00900F5CF72
:1032A00082F4CCEC0AF00900F5CF82F4CCEC0AF001
:1032B0000900F5CF82F4CCEC0AF0D6EC0AF00F90BE
:1032C00097EF19F00401630E826FCCEC0AF0040151
:1032D0002C0E826FCCEC0AF09DEC19F004012C0E40
:1032E000826FCCEC0AF010EC1AF004012C0E826F05
:1032F000CCEC0AF08CEC1AF004012C0E826FCCECB2
:103300000AF00101F80E006FCD0E016F660E026F1C
:10331000030E036FB2EC19F004012C0E826FCCEC9B
:103320000AF0A2EC1AF0D6EC0AF097EF19F00301BC
:10333000C26B07901092A6EF1CF0D8900E0EB3EC63
:1033400007F0E8CF00F10F0EB3EC07F0E8CF01F182
:10335000100EB3EC07F0E8CF02F1110EB3EC07F05A
:10336000E8CF03F10101000E046F000E056F010E9E
:10337000066F000E076F90EC1FF0FDEC1FF02AC1E6
:1033800082F40401300E8227CCEC0AF02BC182F4C7
:103390000401300E8227CCEC0AF02CC182F4040127
:1033A000300E8227CCEC0AF02DC182F40401300EDD
:1033B0008227CCEC0AF02EC182F40401300E822761
:1033C000CCEC0AF02FC182F40401300E8227CCEC41
:1033D0000AF030C182F40401300E8227CCEC0AF0EE
:1033E00031C182F40401300E8227CCEC0AF00401D2
:1033F0002E0E826FCCEC0AF032C182F40401300E42
:103400008227CCEC0AF033C182F40401300E82270B
:10341000CCEC0AF004016D0E826FCCEC0AF01200C5
:10342000120EB3EC07F0E8CF00F1130EB3EC07F087
:10343000E8CF01F1140EB3EC07F0E8CF02F1150E5E
:10344000B3EC07F0E8CF03F101010A0E046F000EA0
:10345000056F000E066F000E076F70EC1FF0000E78
:10346000046F120E056F000E066F000E076F90ECD2
:103470001FF0FDEC1FF02AC182F40401300E8227F8
:10348000CCEC0AF02BC182F40401300E8227CCEC84
:103490000AF02CC182F40401300E8227CCEC0AF031
:1034A0002DC182F40401300E8227CCEC0AF02EC12B
:1034B00082F40401300E8227CCEC0AF02FC182F492
:1034C0000401300E8227CCEC0AF030C182F40401F2
:1034D000300E8227CCEC0AF004012E0E826FCCEC69
:1034E0000AF031C182F40401300E8227CCEC0AF0DC
:1034F00032C182F40401300E8227CCEC0AF033C1D1
:1035000082F40401300E8227CCEC0AF00401730E21
:10351000826FCCEC0AF012000A0EB3EC07F0E8CF91
:1035200000F10B0EB3EC07F0E8CF01F10C0EB3EC99
:1035300007F0E8CF02F10D0EB3EC07F0E8CF03F18E
:10354000C1EF1AF0060EB3EC07F0E8CF00F1070E5A
:10355000B3EC07F0E8CF01F1080EB3EC07F0E8CFC9
:1035600002F1090EB3EC07F0E8CF03F1C1EF1AF056
:1035700001015AEC20F0078457C100F158C101F154
:1035800007940101E80E046F800E056F000E066FB0
:10359000000E076F70EC1FF0000E046F040E056F35
:1035A000000E066F000E076F90EC1FF0880E046F80
:1035B000130E056F000E066F000E076F5FEC1FF015
:1035C0000A0E046F000E056F000E066F000E076FE7
:1035D00090EC1FF0FDEC1FF001012967F5EF1AF0E8
:1035E0000401200E826FF8EF1AF004012D0E826F95
:1035F000CCEC0AF030C182F40401300E8227CCEC0E
:103600000AF031C182F40401300E8227CCEC0AF0BA
:1036100032C182F40401300E8227CCEC0AF004019E
:103620002E0E826FCCEC0AF033C182F40401300E0E
:103630008227CCEC0AF00401430E826FCCEC0AF036
:10364000120087C32AF188C32BF189C32CF18AC3E6
:103650002DF18BC32EF18CC32FF18DC330F18EC3AE
:1036600031F190C332F191C333F10101296BA8EC20
:1036700020F01FEC20F00101000E046F000E056F1A
:10368000010E066F000E076F70EC1FF00E0E0C6E31
:1036900000C10BF09CEC07F00F0E0C6E01C10BF09B
:1036A0009CEC07F0100E0C6E02C10BF09CEC07F0C6
:1036B000110E0C6E03C10BF09CEC07F004017A0EA6
:1036C000826FCCEC0AF004012C0E826FCCEC0AF075
:1036D0000401350E826FCCEC0AF004012C0E826FCF
:1036E000CCEC0AF09DEC19F0A5EF15F087C32AF198
:1036F00088C32BF189C32CF18AC32DF18BC32EF122
:103700008CC32FF18DC330F18EC331F190C332F1F0
:1037100091C333F10101296BA8EC20F01FEC20F0DC
:10372000880E046F130E056F000E066F000E076FF4
:1037300064EC1FF0000E046F040E056F000E066FA0
:10374000000E076F70EC1FF00101E80E046F800E91
:10375000056F000E066F000E076F90EC1FF00A0E4B
:103760000C6E00C10BF09CEC07F00B0E0C6E01C14F
:103770000BF09CEC07F00C0E0C6E02C10BF09CECF5
:1037800007F00D0E0C6E03C10BF09CEC07F004016A
:103790007A0E826FCCEC0AF004012C0E826FCCEC16
:1037A0000AF00401360E826FCCEC0AF004012C0EF4
:1037B000826FCCEC0AF08CEC1AF0A5EF15F087C301
:1037C0002AF188C32BF189C32CF18AC32DF18BC355
:1037D0002EF18CC32FF18DC330F18FC331F190C323
:1037E00032F191C333F10101A8EC20F01FEC20F07D
:1037F000000E046F120E056F000E066F000E076FAD
:1038000070EC1FF001010A0E046F000E056F000E30
:10381000066F000E076F90EC1FF0120E0C6E00C1C9
:103820000BF09CEC07F0130E0C6E01C10BF09CEC3E
:1038300007F0140E0C6E02C10BF09CEC07F0150E95
:103840000C6E03C10BF09CEC07F004017A0E826F42
:10385000CCEC0AF004012C0E826FCCEC0AF00401CF
:10386000370E826FCCEC0AF004012C0E826FCCEC88
:103870000AF010EC1AF0A5EF15F087C32AF188C3FF
:103880002BF189C32CF18AC32DF18BC32EF18CC38C
:103890002FF18DC330F18EC331F190C332F191C35A
:1038A00033F10101296BA8EC20F01FEC20F0880E09
:1038B000046F130E056F000E066F000E076F64ECA9
:1038C0001FF0000E046F040E056F000E066F000E51
:1038D000076F70EC1FF00101E80E046F800E056F9A
:1038E000000E066F000E076F90EC1FF0060E0C6EB8
:1038F00000C10BF09CEC07F0070E0C6E01C10BF041
:103900009CEC07F0080E0C6E02C10BF09CEC07F06B
:10391000090E0C6E03C10BF09CEC07F004017A0E4B
:10392000826FCCEC0AF004012C0E826FCCEC0AF012
:103930000401380E826FCCEC0AF004012C0E826F69
:10394000CCEC0AF0A2EC1AF0A5EF15F081A864EF18
:103950001DF007A81DEF1DF00101800E006F1A0E6B
:10396000016F060E026F000E036F4BC104F14CC1D4
:1039700005F14DC106F14EC107F15FEC1FF003BF29
:1039800064EF1DF0DAEC1DF04BC100F14CC101F108
:103990004DC102F14EC103F107826CEC1EF018C15B
:1039A00004F119C105F11AC106F11BC107F1F80EA6
:1039B000006FCD0E016F660E026F030E036F5FEC9A
:1039C0001FF00E0E0C6E00C10BF09CEC07F00F0EFA
:1039D0000C6E01C10BF09CEC07F0100E0C6E02C1D6
:1039E0000BF09CEC07F0110E0C6E03C10BF09CEC7D
:1039F00007F0078401015AEC20F057C100F158C1CB
:103A000001F107940A0E0C6E00C10BF09CEC07F05C
:103A10000B0E0C6E01C10BF09CEC07F00C0E0C6E43
:103A200002C10BF09CEC07F00D0E0C6E03C10BF005
:103A30009CEC07F0079864EF1DF007AA64EF1DF0F7
:103A4000078401015AEC20F057C100F158C101F17F
:103A50000794060E0C6E00C10BF09CEC07F0070EED
:103A60000C6E01C10BF09CEC07F0080E0C6E02C14D
:103A70000BF09CEC07F0090E0C6E03C10BF09CECF4
:103A800007F0078462C100F163C101F164C102F172
:103A900065C103F10794120E0C6E00C10BF09CEC93
:103AA00007F0130E0C6E01C10BF09CEC07F0140E26
:103AB0000C6E02C10BF09CEC07F0150E0C6E03C1EE
:103AC0000BF09CEC07F0079A0401805181197F0BE1
:103AD0000BE09EA809D014EE00F081517F0BE12687
:103AE000E750812B0F01AD6E05012F51010A13E044
:103AF00081AA8BEF1DF005012F51000A0AE00FB8D3
:103B00008BEF1DF0050130678BEF1DF00FB88BEFC9
:103B10001DF0ACEF29F081B8A0EF1DF095EC22F07C
:103B200005012F51020A02E0A0EF1DF05C2FA0EF6B
:103B30001DF05BC55CF50501010E306F3C0E316F69
:103B400000EC21F030EF0AF018C100F119C101F1C9
:103B50001AC102F11BC103F1000E046F000E056FC4
:103B6000010E066F000E076F90EC1FF029A1CFEF3A
:103B70001DF02051D8B4CFEF1DF018C100F119C1CC
:103B800001F11AC102F11BC103F1000E046F000E16
:103B9000056F0A0E066F000E076F90EC1FF0120003
:103BA000010104510013055101130651021307517D
:103BB000031312000101186B196B1A6B1B6B1200B7
:103BC0002AC182F40401300E8227CCEC0AF02BC10A
:103BD00082F40401300E8227CCEC0AF02CC182F46E
:103BE0000401300E8227CCEC0AF02DC182F40401CE
:103BF000300E8227CCEC0AF02EC182F40401300E84
:103C00008227CCEC0AF02FC182F40401300E822707
:103C1000CCEC0AF030C182F40401300E8227CCECE7
:103C20000AF031C182F40401300E8227CCEC0AF094
:103C300032C182F40401300E8227CCEC0AF033C189
:103C400082F40401300E8227CCEC0AF012002FC15E
:103C500082F40401300E8227CCEC0AF030C182F4E9
:103C60000401300E8227CCEC0AF031C182F4040149
:103C7000300E8227CCEC0AF032C182F40401300EFF
:103C80008227CCEC0AF033C182F40401300E822783
:103C9000CCEC0AF01200060E116E060E126E060E25
:103CA000136E112E51EF1EF0122E51EF1EF0132E37
:103CB00051EF1EF08B84020E116E020E126E020E78
:103CC000136E112E61EF1EF0122E61EF1EF0132EF7
:103CD00061EF1EF08B9412000101005305E10153C6
:103CE00003E1025301E1002B2FEC1FF05AEC20F00E
:103CF0003951006F3A51016F420E046F4B0E056F40
:103D0000000E066F000E076F70EC1FF000C104F18B
:103D100001C105F102C106F103C107F118C100F1AB
:103D200019C101F11AC102F11BC103F107B29DEFE4
:103D30001EF064EC1FF09FEF1EF05FEC1FF000C15F
:103D400018F101C119F102C11AF103C11BF11200EE
:103D50005AEC20F059C100F15AC101F1060EB3EC42
:103D600007F0E8CF04F1070EB3EC07F0E8CF05F158
:103D7000080EB3EC07F0E8CF06F1090EB3EC07F03C
:103D8000E8CF07F15FEC1FF000C124F101C125F17C
:103D900002C126F103C127F1290E046F000E056F41
:103DA000000E066F000E076F70EC1FF0EE0E046F32
:103DB000430E056F000E066F000E076F64EC1FF0D8
:103DC00024C104F125C105F126C106F127C107F17F
:103DD00070EC1FF000C11CF101C11DF102C11EF108
:103DE00003C11FF1120EB3EC07F0E8CF04F1130E7C
:103DF000B3EC07F0E8CF05F1140EB3EC07F0E8CF11
:103E000006F1150EB3EC07F0E8CF07F10D0E006FC9
:103E1000000E016F000E026F000E036F70EC1FF0BA
:103E2000180E046F000E056F000E066F000E076F70
:103E300090EC1FF01CC104F11DC105F11EC106F17B
:103E40001FC107F164EC1FF06A0E046F2A0E056FA4
:103E5000000E066F000E076F5FEC1FF01200BF0E22
:103E6000FA6E200E3A6F396BD8900037013702375F
:103E70000337D8B040EF1FF03A2F35EF1FF0390766
:103E80003A070353D8B412000331070B80093F6F80
:103E900003390F0B010F396F80EC5FF0406F39056C
:103EA00080EC5FF0405D405F396B3F33D8B039271D
:103EB00039333FA955EF1FF0405139271200010156
:103EC0007FEC20F0D8B01200010103510719346FC4
:103ED00042EC20F0D8900751031934AF800F120044
:103EE0000101346B66EC20F0D8A07CEC20F0D8B057
:103EF000120051EC20F05AEC20F01F0E366F92ECBD
:103F000020F00B35D8B042EC20F0D8A00335D8B063
:103F10001200362F7FEF1FF034B169EC20F0120051
:103F20000101346B04510511061107110008D8A0D6
:103F300066EC20F0D8A07CEC20F0D8B01200086B22
:103F4000096B0A6B0B6B92EC20F01F0E366F92EC34
:103F500020F007510B5DD8A4BAEF1FF006510A5D9F
:103F6000D8A4BAEF1FF00551095DD8A4BAEF1FF02D
:103F70000451085DD8A0CDEF1FF00451085F055132
:103F8000D8A0053D095F0651D8A0063D0A5F07513C
:103F9000D8A0073D0B5FD8900081362FA7EF1FF008
:103FA00034B169EC20F0346B66EC20F0D89096ECDC
:103FB00020F007510B5DD8A4EAEF1FF006510A5D0F
:103FC000D8A4EAEF1FF00551095DD8A4EAEF1FF06D
:103FD0000451085DD8A0F9EF1FF0003FF9EF1FF082
:103FE000013FF9EF1FF0023FF9EF1FF0032BD8B4A8
:103FF000120034B169EC20F012000101346B66EC60
:1040000020F0D8B012009BEC20F0200E366F003765
:1040100001370237033711EE33F00A0E376FE736F8
:104020000A0EE75CD8B0E76EE552372F0FEF20F0AD
:10403000362F07EF20F034B12981D890120001010A
:104040000A0E346F200E366F11EE29F03451376F9F
:104050000A0ED890E652D8B0E726E732372F2AEF7B
:1040600020F00333023301330033362F24EF20F0E6
:10407000E750FF0FD8A00335D8B0120029B169EC82
:1040800020F01200045100270551D8B0053D01274A
:104090000651D8B0063D02270751D8B0073D032787
:1040A00012000051086F0151096F02510A6F03514C
:1040B0000B6F12000101006B016B026B036B1200AE
:1040C0000101046B056B066B076B12000335D8A06A
:1040D00012000351800B001F011F021F031F003F2E
:1040E00079EF20F0013F79EF20F0023F79EF20F0E7
:1040F000032B342B032512000735D8A012000751DB
:10410000800B041F051F061F071F043F8FEF20F0C1
:10411000053F8FEF20F0063F8FEF20F0072B342B69
:1041200007251200003701370237033708370937F0
:104130000A370B3712000101296B2A6B2B6B2C6B92
:104140002D6B2E6B2F6B306B316B326B336B120020
:1041500001012A510F0B2A6F2B510F0B2B6F2C5182
:104160000F0B2C6F2D510F0B2D6F2E510F0B2E6F30
:104170002F510F0B2F6F30510F0B306F31510F0B31
:10418000316F32510F0B326F33510F0B336F1200FF
:104190008A96400EC76E200EC66E9E96CC0EC96ED5
:1041A0009EA6D0EF20F09E960B0EC96E9EA6D6EF6F
:1041B00020F08A860F8412008A96400EC76E200E69
:1041C000C66E9E96000EC96E9EA6E4EF20F09E96E7
:1041D000000EC96E9EA6EAEF20F08A868A969E9609
:1041E000820EC96E9EA6F2EF20F09E96C3C3C9FF51
:1041F0009EA6F8EF20F081B2FBEF20F08A86120035
:1042000081B2E3EF21F08A96400EC76E200EC66E93
:104210009E96000EC96E9EA60BEF21F0C9AEE3EF8D
:1042200021F09E96000EC96E9EA614EF21F0C9CF14
:10423000E8FF240A07E10F8600C504F501C505F56E
:104240000501066B0FA657EF21F005010501065188
:10425000010A16E005010651020A16E005010651A1
:10426000030A16E005010651040A16E0050106518D
:10427000050A16E005010651090A16E056EF21F07D
:10428000C9CF07F556EF21F0C9CF08F556EF21F059
:10429000C9CF09F556EF21F0C9CF0AF556EF21F045
:1042A000C9CF0BF556EF21F0C9CF0CF5062BC9CFBE
:1042B000E8FF0A0A77E10F9605010751470A72E104
:1042C00005010951470A12E005010951520A52E05D
:1042D00005010951560A56E0050109514D0A58E0F9
:1042E000050109515A0A5AE0D2EF21F005010A519D
:1042F000470A1CE005010A514C0A1EE005010B515A
:10430000410A20E005010B51560A02E0D2EF21F0EC
:1043100005010C51310A1CE005010C51320A1EE066
:1043200005010C51330A20E0D2EF21F004C50DF550
:1043300005C50EF5D2EF21F004C50FF505C510F542
:10434000D2EF21F004C511F505C512F5D2EF21F029
:1043500004C513F505C514F5D2EF21F004C515F514
:1043600005C516F5D2EF21F004C517F505C518F5FA
:10437000D2EF21F004C519F505C51AF5CFEC27F0E9
:10438000D2EF21F004C51BF505C51CF5D2EF21F0D5
:1043900004C51DF505C51EF5D2EF21F004C51FF5B6
:1043A00005C520F527EE00F005010051D926015181
:1043B000D8B00129DA26C9CFDFFF0501012B003F64
:1043C0000107030E01178A8612008984000EC76E4A
:1043D000220EC66E9E96C69E000EC96EFF0E9EB63B
:1043E00002D0E82EFCD79E96C69E000EC96EFF0E28
:1043F0009EB602D0E82EFCD7C9CFABF59E96C69EDE
:10440000000EC96EFF0E9EB602D0E82EFCD7C9CFB3
:10441000ACF59E96C69E000EC96EFF0E9EB602D0EB
:10442000E82EFCD7C9CFADF59E96C69E000EC96E8C
:10443000FF0E9EB602D0E82EFCD7C9CFAEF59E96F1
:10444000C69E000EC96EFF0E9EB602D0E82EFCD7A7
:10445000C9CFAFF59E96C69E000EC96EFF0E9EB6E2
:1044600002D0E82EFCD7C9CFB0F59E96C69E000EAE
:10447000C96EFF0E9EB602D0E82EFCD7C9CFB1F5AB
:10448000899498EC24F012008984000EC76E220EE5
:10449000C66E9E96C69E800EC96EFF0E9EB602D058
:1044A000E82EFCD79E96C69EABC5C9FFFF0E9EB6F2
:1044B00002D0E82EFCD79E96C69EACC5C9FFFF0E63
:1044C0009EB602D0E82EFCD79E96C69EADC5C9FF0B
:1044D000FF0E9EB602D0E82EFCD79E96C69EAEC5B5
:1044E000C9FFFF0E9EB602D0E82EFCD79E96C69E50
:1044F000AFC5C9FFFF0E9EB602D0E82EFCD79E9630
:10450000C69EB0C5C9FFFF0E9EB602D0E82EFCD7EE
:104510009E96C69EB1C5C9FFFF0E9EB602D0E82E7C
:10452000FCD7899498EC24F012008984000EC76EA1
:10453000220EC66E9E96C69E070EC96EFF0E9EB6D2
:1045400002D0E82EFCD79E96C69E000EC96EFF0EC6
:104550009EB602D0E82EFCD7C9CFABF59E96C69E7C
:10456000000EC96EFF0E9EB602D0E82EFCD7C9CF52
:10457000ACF59E96C69E000EC96EFF0E9EB602D08A
:10458000E82EFCD7C9CFADF59E96C69E000EC96E2B
:10459000FF0E9EB602D0E82EFCD7C9CFAEF58994A7
:1045A00098EC24F08984000EC76E220EC66E9E968B
:1045B000C69E0F0EC96EFF0E9EB602D0E82EFCD727
:1045C0009E96C69E000EC96EFF0E9EB602D0E82EC5
:1045D000FCD7C9CFB3F5899498EC24F012008984F4
:1045E000000EC76E220EC66E9E96C69E870EC96EC0
:1045F000FF0E9EB602D0E82EFCD79E96C69EABC597
:10460000C9FFFF0E9EB602D0E82EFCD79E96C69E2E
:10461000ACC5C9FFFF0E9EB602D0E82EFCD79E9611
:10462000C69EADC5C9FFFF0E9EB602D0E82EFCD7D0
:104630009E96C69EAEC5C9FFFF0E9EB602D0E82E5E
:10464000FCD7899498EC24F089849E96C69E8F0EA0
:10465000C96EFF0E9EB602D0E82EFCD79E96C69E6F
:10466000B3C5C9FFFF0E9EB602D0E82EFCD78994D1
:1046700098EC24F012008984000EC76E220EC66EDC
:104680009E96C69E870EC96EFF0E9EB602D0E82E7D
:10469000FCD79E96C69E000EC96EFF0E9EB602D037
:1046A000E82EFCD79E96C69E800EC96EFF0E9EB663
:1046B00002D0E82EFCD79E96C69E800EC96EFF0ED5
:1046C0009EB602D0E82EFCD79E96C69E800EC96E7E
:1046D000FF0E9EB602D0E82EFCD7899498EC24F009
:1046E00089849E96C69E8F0EC96EFF0E9EB602D01E
:1046F000E82EFCD79E96C69E010EC96EFF0E9EB692
:1047000002D0E82EFCD7899498EC24F0120089841A
:10471000000EC76E220EC66E9E96C69E870EC96E8E
:10472000FF0E9EB602D0E82EFCD79E96C69E000EC7
:10473000C96EFF0E9EB602D0E82EFCD79E96C69E8E
:10474000000EC96EFF0E9EB602D0E82EFCD79E96D4
:10475000C69E800EC96EFF0E9EB602D0E82EFCD714
:104760009E96C69E800EC96EFF0E9EB602D0E82EA3
:10477000FCD7899498EC24F089849E96C69E8F0E6F
:10478000C96EFF0E9EB602D0E82EFCD79E96C69E3E
:10479000010EC96EFF0E9EB602D0E82EFCD789949A
:1047A00098EC24F012008984000EC76E220EC66EAB
:1047B0009E96C69E8F0EC96EFF0E9EB602D0E82E44
:1047C000FCD798EC24F09E96C69E810EC96EFF0E13
:1047D0009EB602D0E82EFCD7899498EC24F0898408
:1047E000000EC76E220EC66E9E96C69E8F0EC96EB6
:1047F000FF0E9EB602D0E82EFCD798EC24F09E96D1
:10480000C69E010EC96EFF0E9EB602D0E82EFCD7E2
:10481000899498EC24F089849E96C69E910EC96E68
:10482000FF0E9EB602D0E82EFCD798EC24F09E96A0
:10483000C69EA50EC96EFF0E9EB602D0E82EFCD70E
:10484000899498EC24F012008984000EC76E220E21
:10485000C66E9E96C69E8F0EC96EFF0E9EB602D085
:10486000E82EFCD798EC24F09E96C69E810EC96E69
:10487000FF0E9EB602D0E82EFCD7899498EC24F067
:1048800012008984000EC76E220EC66E9E96C69ECA
:104890008F0EC96EFF0E9EB602D0E82EFCD798ECA4
:1048A00024F09E96C69E010EC96EFF0E9EB602D0E3
:1048B000E82EFCD7899498EC24F012008984000E2D
:1048C000C76E220EC66E9E96C69E910EC96EFF0ED4
:1048D0009EB602D0E82EFCD798EC24F09E96C69E99
:1048E000A50EC96EFF0E9EB602D0E82EFCD78994A5
:1048F00098EC24F012008984000EC76E220EC66E5A
:104900009E96C69E910EC96EFF0E9EB602D0E82EF0
:10491000FCD798EC24F09E96C69E000EC96EFF0E42
:104920009EB602D0E82EFCD7899498EC24F01200B1
:10493000050EE82EFED712000501256B266B276BAE
:10494000286B899A400EC76E200EC66E9E96C69E34
:10495000030EC96EFF0E9EB602D0E82EFCD79E96BF
:10496000C69E27C5C9FFFF0E9EB602D0E82EFCD713
:104970009E96C69E26C5C9FFFF0E9EB602D0E82EA3
:10498000FCD79E96C69E25C5C9FFFF0E9EB602D0D7
:10499000E82EFCD79E96C69EC952FF0E9EB602D048
:1049A000E82EFCD7898A0F01C950FF0A01E11200E5
:1049B00005012E51130A05E005012E51170A0CE0DE
:1049C00012000501F00E256FFF0E266F0F0E276FE8
:1049D000000E286FF5EF24F00501F00E256FFF0E95
:1049E000266FFF0E276F000E286F899A400EC76E44
:1049F000200EC66E9E96C69E030EC96EFF0E9EB614
:104A000002D0E82EFCD79E96C69E27C5C9FFFF0E92
:104A10009EB602D0E82EFCD79E96C69E26C5C9FF3C
:104A2000FF0E9EB602D0E82EFCD79E96C69E25C5E8
:104A3000C9FFFF0E9EB602D0E82EFCD79E96C69EFA
:104A4000C952FF0E9EB602D0E82EFCD7898A0F010C
:104A5000C950FF0A1EE005012E51130A05E00501A9
:104A60002E51170A0CE012000501000E256F000EF2
:104A7000266F100E276F000E286FF5EF24F005014A
:104A8000000E256F000E266F000E276F010E286F97
:104A900012000501256B266B276B286B05012E5133
:104AA000130A05E005012E51170A0CE0120005015A
:104AB000000E216F000E226F040E236F000E246F74
:104AC0006BEF25F00501000E216F000E226F800EA6
:104AD000236F000E246F21C500F122C501F123C50B
:104AE00002F124C503F125C504F126C505F127C54A
:104AF00006F128C507F1D0EC1DF000C125F501C174
:104B000026F502C127F503C128F5899A400EC76E24
:104B1000200EC66E9E96C69E030EC96EFF0E9EB6F2
:104B200002D0E82EFCD79E96C69E27C5C9FFFF0E71
:104B30009EB602D0E82EFCD79E96C69E26C5C9FF1B
:104B4000FF0E9EB602D0E82EFCD79E96C69E25C5C7
:104B5000C9FFFF0E9EB602D0E82EFCD79E96C69ED9
:104B6000C952FF0E9EB602D0E82EFCD7898AC950E2
:104B7000FF0A08E104C125F505C126F506C127F5A0
:104B800007C128F5D890050124332333223321337C
:104B90002151F00B216F2167D5EF25F02267D5EF6A
:104BA00025F02367D5EF25F024676BEF25F005018D
:104BB000100E2527E86A2623E86A2723E86A2823B7
:104BC0001200E86A05012E51130A06E005012E5174
:104BD000170A0BE0020E120005012851000A03E13A
:104BE0002751F00B07E0010E120005012851000AC1
:104BF00001E0010E120029C500F12AC501F12BC503
:104C000002F12CC503F125C504F126C505F127C520
:104C100006F128C507F15FEC1FF003BF1200E1ECBD
:104C200025F05FE1899A400EC76E200EC66E9E96F3
:104C3000C69E060EC96EFF0E9EB602D0E82EFCD7A9
:104C4000898A899A9E96C69E020EC96EFF0E9EB6EE
:104C500002D0E82EFCD79E96C69E27C5C9FFFF0E40
:104C60009EB602D0E82EFCD79E96C69E26C5C9FFEA
:104C7000FF0E9EB602D0E82EFCD79E96C69E25C596
:104C8000C9FFFF0E9EB602D0E82EFCD79E96C69EA8
:104C9000000EC96EFF0E9EB602D0E82EFCD7898AA0
:104CA000899A9E96C69E050EC96EFF0E9EB602D0CC
:104CB000E82EFCD79E96C69EC952FF0E9EB602D025
:104CC000E82EFCD7C9B05AEF26F0898A0501100EEC
:104CD0002527E86A2623E86A2723E86A2823FBEFCA
:104CE00025F01200899A400EC76E200EC66E9E9661
:104CF000C69E060EC96EFF0E9EB602D0E82EFCD7E9
:104D0000898A899A9E96C69EC70EC96EFF0E9EB668
:104D100002D0E82EFCD7898A0501256B266B276B0C
:104D2000286B1200899A400EC76E200EC66E9E96A2
:104D3000C69E050EC96EFF0E9EB602D0E82EFCD7A9
:104D40009E96C69EC952FF0E9EB602D0E82EFCD794
:104D5000C9CF33F5898A1200899A400EC76E200E9A
:104D6000C66E9E96C69EB90EC96EFF0E9EB602D046
:104D7000E82EFCD7898A1200899A400EC76E200E51
:104D8000C66E9E96C69EAB0EC96EFF0E9EB602D034
:104D9000E82EFCD7898AFF0EE82EFED71200E1EC40
:104DA00025F0D8A41200899A400EC76E200EC66E58
:104DB0009E96C69E030EC96EFF0E9EB602D0E82ECA
:104DC000FCD79E96C69E27C5C9FFFF0E9EB602D091
:104DD000E82EFCD79E96C69E26C5C9FFFF0E9EB63E
:104DE00002D0E82EFCD79E96C69E25C5C9FFFF0EB1
:104DF0009EB602D0E82EFCD79E96C69EC952FF0EE4
:104E00009EB602D0E82EFCD7898A0F01C950FF0A4E
:104E1000D8A4CEEF27F00501FE0E336F0501000E7A
:104E2000336FE5EC21F0ABC534F5ACC535F5ADC558
:104E300036F5AEC537F5AFC538F5B0C539F5B1C5EE
:104E40003AF50784B6C166F1B7C167F1B8C168F138
:104E5000B9C169F14BC14FF14CC150F14DC151F194
:104E60004EC152F157C159F158C15AF10794CFECD4
:104E700015F000C13BF501C13CF502C13DF503C190
:104E80003EF505015D674CEF27F05E674CEF27F0BC
:104E90005F674CEF27F0606750EF27F05EEF27F079
:104EA0005DC504F15EC505F15FC506F160C507F19A
:104EB00001015FEC1FF003BFCEEF27F059C13FF5B2
:104EC0005AC140F5B5C541F5B6C542F50501100E0C
:104ED000326F899A400EC76E200EC66E9E96C69E91
:104EE000060EC96EFF0E9EB602D0E82EFCD7898A48
:104EF000899A9E96C69E020EC96EFF0E9EB602D07D
:104F0000E82EFCD79E96C69E27C5C9FFFF0E9EB60B
:104F100002D0E82EFCD79E96C69E26C5C9FFFF0E7E
:104F20009EB602D0E82EFCD79E96C69E25C5C9FF28
:104F3000FF0E9EB602D0E82EFCD725EE33F0322FBE
:104F400002D0AEEF27F09E96C69EDECFC9FFFF0EC1
:104F50009EB602D0E82EFCD79FEF27F0898A899A67
:104F60009E96C69E050EC96EFF0E9EB602D0E82E16
:104F7000FCD79E96C69EC952FF0E9EB602D0E82E62
:104F8000FCD7C9B0B9EF27F0898A0501100E252793
:104F9000E86A2623E86A2723E86A2823120019C54D
:104FA00002F51AC503F525EE65F00501326B17EE23
:104FB00000F005010251E1260351D8B00329E22691
:104FC000E7CFE8FF2C0A06E132C5DEFF0501326BB0
:104FD000F2EF27F0E7CFE8FF2A0A0CE0E7CFDEFF89
:104FE0000501322B0501032B023F0307030E0317B4
:104FF000D7EF27F00501336B346B356B366B376BAE
:10500000386B396B3A6B3B6B3C6B3D6B3E6B3F6B6C
:10501000406B416B426B436B446B456B466B476B1C
:10502000486B496B4A6B4B6B4C6B4D6B4E6B4F6BCC
:10503000506B516B526BDDCFE8FF0501325105E03B
:10504000DDCFE8FF322F20EF28F00501DDCF32F56C
:10505000325105E0DDCFE8FF322F2AEF28F00501BD
:10506000DDCF32F5325105E0DDCFE8FF322F34EFEE
:1050700028F011EE33F001019BEC20F00501DDCFAB
:1050800032F5325105E0DDCFE5FF322F43EF28F056
:105090000101A8EC20F01FEC20F000C134F501C1A3
:1050A00035F502C136F50501DDCF32F5325105E0A7
:1050B000DDCFE8FF322F58EF28F00501DDCF32F5C4
:1050C000325105E0DDCFE8FF322F62EF28F0050115
:1050D000DDCF32F5325107E0DDCFE8FFE8A83385B8
:1050E000322F6CEF28F011EE33F001019BEC20F031
:1050F0000501DDCF32F5325114E0DDCFE5FFDDCF24
:10510000E5FFDDCFE5FFDDCFE5FFDDCFE8FFDDCF5C
:10511000E5FFDDCFE5FFDDCFE5FFDDCFE5FFDDCF4F
:10512000E5FF0101A8EC20F01FEC20F000C13EF5E6
:1051300001C13FF502C140F503C141F50501DDCFD5
:1051400032F5325107E0DDCFE8FFE8A83383322F94
:10515000A3EF28F011EE33F001019BEC20F00501E4
:10516000DDCF32F5325105E0DDCFE5FF322FB4EF70
:1051700028F001012EC12FF12DC12EF12CC12DF1EE
:105180002BC12CF1A8EC20F01FEC20F000C13AF567
:1051900001C13BF502C13CF503C13DF50501DDCF81
:1051A00032F5325107E0DDCFE8FF322FD3EF28F0A0
:1051B000E8B0338711EE33F001019BEC20F0DDCF36
:1051C000E8FFDDCFE8FFDDCFE8FFDDCFE8FFDDCF93
:1051D000E8FFDDCFE5FFDDCFE5FFDDCFE5FFDDCF8C
:1051E000E5FFDDCFE5FFDDCFE5FFA8EC20F01FEC0C
:1051F00020F000C137F501C138F502C139F5078447
:1052000062C166F163C167F164C168F165C169F1AA
:105210004BC14FF14CC150F14DC151F14EC152F152
:1052200057C159F158C15AF10794CFEC15F000C19C
:1052300042F501C143F502C144F503C145F5120031
:1052400021C500F122C501F123C502F124C503F1F6
:10525000899A400EC76E200EC66E9E96C69E0B0E95
:10526000C96EFF0E9EB602D0E82EFCD79E96C69E53
:1052700002C1C9FFFF0E9EB602D0E82EFCD79E9653
:10528000C69E01C1C9FFFF0E9EB602D0E82EFCD714
:105290009E96C69E00C1C9FFFF0E9EB602D0E82EA4
:1052A000FCD79E96C69EC952FF0E9EB602D0E82E2F
:1052B000FCD725EE33F00501100E326F9E96C69E88
:1052C000C952FF0E9EB602D0E82EFCD7C9CFDEFF32
:1052D000322F5EEF29F0898A1200899A400EC76E3C
:1052E000200EC66E9E96C69E900EC96EFF0E9EB68E
:1052F00002D0E82EFCD79E96C69E000EC96EFF0E09
:105300009EB602D0E82EFCD79E96C69E000EC96EB1
:10531000FF0E9EB602D0E82EFCD79E96C69E000ECB
:10532000C96EFF0E9EB602D0E82EFCD79E96C69E92
:10533000C952FF0E9EB602D0E82EFCD7C9CF2DF57C
:105340009E96C69EC952FF0E9EB602D0E82EFCD78E
:10535000C9CF2EF5898A12004BEC1EF0B5C5E8FFC7
:10536000D70802E34BEC1EF0B5C5E8FFC80802E31E
:105370004BEC1EF0B5C5E8FFB90802E34BEC1EF09C
:10538000B5C5E8FFAA0802E34BEC1EF0B5C5E8FF7F
:105390009B0802E34BEC1EF095EC22F0ACEC26F0FF
:1053A000F29CF29E8B948A86C69AC2908A949482CA
:1053B000948C720ED36ED3A4FED789968A90939064
:1053C000FF0EE8CF00F0E82EFED7002EFCD781506C
:1053D000F294F29A9E909D909E929D92F298F292F3
:0A53E000F290F286F28E0300FF0047
:10BF0000E844F926000C160C2B0C3F0C520C640C68
:10BF1000760C860C960CA50CB30CC10CCF0CDC0C6B
:06BF2000E80CF40C000C1B
:00000001FF
